:100000000C947C020C94B4020C94B4020C94B402D0
:100010000C94B4020C94B4020C94B4020C94B40288
:100020000C94B4020C94B4020C94B4020C94762593
:100030000C9425260C9488200C94B4020C94B402E1
:100040000C94B4020C94B4020C94B4020C941021DD
:100050000C94B4020C94B4020C94B4020C94B40248
:100060000C94B4020C94B4020C94B4020C94B40238
:100070000C94B402D205D205FE05FE056606840680
:100080009C079C078F062807390739079226B9264F
:10009000B127B926B12705272827B1277F278E2723
:1000A000680069006A416B006C006D00C35CC45C51
:1000B0000100C65CCA5C0251005CC55C0000C75C04
:1000C000CB5C010000000000000000002A2B28008B
:1000D00000000000000000000000000000000029F7
:1000E000000000002C1E3420212224342627252E37
:1000F000362D3738271E1F2021222324252633336F
:10010000362E37381F0405060708090A0B0C0D0E9A
:100110000F101112131415161718191A1B1C1D2F66
:100120003130232D350405060708090A0B0C0D0E86
:100130000F101112131415161718191A1B1C1D2F46
:100140003130354C000000000000000000000000CD
:10015000000000000000000000000000000000009F
:1001600000000000000000007E0F00D4FFFFFFC76A
:10017000000000787F3F1F643214643214783C1E04
:100180001E140A052223252628292A2C2D2F303239
:10019000333536383A3B3D3E4042434547494A4C69
:1001A0004E5051535557595A5C5E60626466686997
:1001B0006B6D6F71737577797B7D7F81838587899F
:1001C0008A8C8E90929496989A9C9E9FA1A3A5A7A4
:1001D000A8AAACAEAFB1B3B4B6B8B9BBBCBEBFC1D0
:1001E000C2C3C5C6C7C9CACBCCCDCED0D1D2D2D35B
:1001F000D4D5D6D7D7D8D9D9DADADBDBDBDCDCDC6F
:10020000DCDCDDDDDDDDDCDCDCDCDCDBDBDBDADA31
:10021000D9D9D8D7D7D6D5D4D3D2D2D1D0CECDCCA8
:10022000CBCAC9C7C6C5C3C2C1BFBEBCBBB9B8B6BD
:10023000B4B3B1AFAEACAAA8A7A5A3A19F9E9C9A48
:1002400098969492908E8C8A89878583817F7D7B16
:1002500079777573716F6D6B6968666462605E5CF7
:100260005A5957555351504E4C4A494745434240BD
:100270003E3D3B3A3836353332302F2D2C2A292853
:1002800026252322FFAA7F5540000101010101011B
:10029000010101020202020202020202030303033D
:1002A000030303030404040404040405050505050D
:1002B00006060606060707070707080808080909CB
:1002C00009090A0A0A0B0B0B0C0C0C0D0D0D0E0E76
:1002D0000E0F0F0F10101111111212131314141509
:1002E0001516161717181819191A1A1B1B1C1D1D7D
:1002F0001E1E1F20202122222324242526262728D3
:1003000029292A2B2C2D2D2E2F3031323233343502
:10031000363738393A3B3C3D3E3F40414243444505
:10032000464748494A4C4D4E4F50515354555658E4
:10033000595A5B5D5E5F616264656668696B6C6D8E
:100340006F7072737577787A7B7D7E808283858704
:10035000888A8C8E8F91939596989A9C9EA0A2A342
:10036000A5A7A9ABADAFB1B3B5B7BABCBEC0C2C447
:10037000C6C9CBCDCFD1D4D6D8DBDDDFE2E4E7E907
:10038000EBEEF0F3F5F8FAFDFF0E0336006D0061B9
:1003900000630072006F00000016036A006F0061C6
:1003A000006F00660062006D00610069006100007E
:1003B000000403090409023B00020100A0FA090439
:1003C0000000010301010009211101000122400088
:1003D0000705810308000109040100010300000072
:1003E00009211101000122B6000705820320000146
:1003F0001201000200000008EDFE370001000102BA
:10040000000105010902A10185020901A1000509F8
:1004100019012908150025019508750181020501BA
:10042000093009311581257F950275088106093843
:100430001581257F950175088106050C0A3802157E
:1004400081257F950175088106C0C005010980A13D
:1004500001850319012AB700150126B7009501751A
:10046000108100C0050C0901A101850419012AA011
:1004700002150126A002950175108100C005010931
:1004800006A1018506050719E029E7150025019554
:1004900008750181020507190029EF15002501954E
:1004A000F07501810205081901290595057501916D
:1004B00002950175039101C005010906A101050717
:1004C00019E029E7150025019508750181029501BC
:1004D000750881010507190029FF150026FF009501
:1004E0000675088100050819012905950575019112
:1004F00002950175039101C011241FBECFEFD4E016
:10050000DEBFCDBF04B603FE18C08091D902909122
:10051000DA02A091DB02B091DC028730904BA74059
:10052000B04B59F41092D9021092DA021092DB0209
:100530001092DC02E0E0F8E3099511E0A0E0B1E000
:10054000E6E5F1E502C005900D92A43BB107D9F7AD
:1005500022E0A4EBB1E001C01D92A93DB207E1F792
:100560000E9456130C94A9280C9400009C013A9503
:1005700021153F4130F5BC0166277270AC0144275C
:1005800054709C012227387094FF0FC090FF02C066
:1005900080E101C080E0672B09F08062452B09F003
:1005A0008064232B79F080680895892F8170672BF0
:1005B00009F08260452B09F08460232B19F08860D4
:1005C000089580E00895CF93DF93EB010E94B60277
:1005D000FE01DF91CF910994CF93DF93EC01805E10
:1005E0009109089710F0209719F469E875E002C0A6
:1005F00064E178E0CE010E94E3028C2FDF91CF917D
:100600000C94DF04CF93DF93EC010E943505CE01FB
:10061000805E9109089710F0209719F460E975E061
:1006200002C06BE178E0CE01DF91CF910C94E30240
:10063000CF93DF93EC010E94EC02C933D10549F45A
:100640002FEF87EE93E0215080409040E1F700C00B
:100650000000CE01DF91CF910C94020381E0089558
:1006600081E008950C94300308950C9434031F9393
:10067000CF93DF9300D000D01F92CDB7DEB7498370
:100680005A836B833091B70189819A81311114C0EB
:10069000662359F0222349F00E94EC09182F682F95
:1006A00089819A810E94900903C00E94BF09182F76
:1006B00069817A81812F04C00E94EC0969817A8165
:1006C0000F900F900F900F900F90DF91CF911F918F
:1006D0000C940C11FC01262F4081518162817381A1
:1006E00084810C94370381E00895CF93DF93EC016C
:1006F00060E00E946A03BE01DF91CF910C94350344
:100700000C9440120C943C1208950E943A080E94E6
:1007100084032FEF84E39CE0215080409040E1F778
:1007200000C000000C9436210F931F93CF93DF93EA
:100730008C0161E00E946A03EC01B8010E9432035F
:10074000882309F44BC0B801CE010E94C51C882340
:1007500009F444C0B801CE010E94CF1E8823F1F1F4
:10076000B801CE010E94E31C8823C1F1B801CE017B
:100770000E942B1E882391F1B801CE010E94031B19
:10078000882361F1F8018281882309F1CB358DE559
:10079000D807C1F050F4C115FCE5DF0781F0CF3D6B
:1007A000DC45A9F40E941C0F19C0CC35EDE5DE072D
:1007B00061F0CD35DD4559F40E94650E08C00E94F8
:1007C00085030CC00E946E0E02C00E94710EC8010B
:1007D000DF91CF911F910F910C942E0380E0DF9158
:1007E000CF911F910F9108950E9469200C947D0470
:1007F0000E9480040C946F20DF92EF92FF920F937F
:100800001F93CF93DF93E82FF0E0EC53FF4FD4908A
:10081000282F26952695269530E0F901EC59FE4FB4
:100820000491877010E0082E02C0159507950A9470
:10083000E2F701701127F901EC5AFE4FE490F12C18
:10084000082E02C0F594E7940A94E2F791E0E922B9
:10085000FF24F901EC5BFE4FC491D0E002C0D595B6
:10086000C7958A95E2F7C170DD270115110519F0CA
:1008700081EE0E94DF04E114F10419F086EE0E947B
:10088000DF048D2D0E948005EF2819F086EE0E946E
:100890003505012B19F081EE0E943505CD2B51F065
:1008A0008CE2DF91CF911F910F91FF90EF90DF903D
:1008B0000C948005DF91CF911F910F91FF90EF90E5
:1008C000DF900895982F9F709A50963010F0805DB9
:1008D00001C0895A0C94FC0308950C946C0481E0C7
:1008E00008950C946F040895CF93C82F0E946D044F
:1008F0008C2F0E947104CF91089580E00C947404B1
:100900000E942B1F0C9474040E942B1F9091B6011F
:10091000891721F08093B6010C9474040895CF9345
:10092000DF93CDB7DEB72B970FB6F894DEBF0FBEBF
:10093000CDBF4F83588769877A878B8761110E9463
:10094000B10D9E012F5F3F4F86E0F90111928A950C
:10095000E9F785E0FE013796D90101900D928A955D
:10096000E1F789819A814C815D81452B31F09F3F70
:1009700031F491E08F3F19F403C091E001C090E0A1
:1009800090FF09C049815A816B817C818D819E8154
:100990000E94CA0C05C0C9010E9473038111F2CFE5
:1009A0002B960FB6F894DEBF0FBECDBFDF91CF916F
:1009B0000895FC01808191810E942E0A0895CF93B1
:1009C000882309F450C0C82F8CEF8C0F813AD0F4E3
:1009D0006C2F80910201909103010E94A41F882333
:1009E00049F06C2F80910201909103010E942F2009
:1009F0000E94D30D6C2F80910201909103010E94FF
:100A000024200CC080E28C0F883058F4C77081E03D
:100A100001C0880FCA95EAF70E94910DCF910C94FE
:100A2000D30DEBE5EC0FE33040F4F0E0E75AFE4F76
:100A3000808190E0CF910C94621FE8E5EC0FE731E4
:100A400050F4F0E0EE0FFF1FE55DFE4F80819181D5
:100A5000CF910C94781FCD3E30F08C2F0E94E31381
:100A6000CF910C94B514CF910895882389F19CEF10
:100A7000980F913A40F4682F809102019091030100
:100A80000E942F200DC090E2980F983058F4877084
:100A900091E001C0990F8A95EAF7892F0E94970D7E
:100AA0000C94D30D9BE5980F933020F480E090E0F8
:100AB0000C94621F98E5980F973120F480E090E045
:100AC0000C94781F8D3E20F00E943E140C94B514B7
:100AD00008951F93CF93DF93182FEB010E94DF043B
:100AE000209741F08FE99FE00197F1F700C00000E7
:100AF0002197F6CF812FDF91CF911F910C9435056F
:100B0000893319F060E070E002C060E570E00C9499
:100B10006905882321F00E94910D0C94D30D08954E
:100B2000882321F00E94970D0C94D30D0895CF9245
:100B3000DF92EF92FF920F931F93CF93DF937C018D
:100B4000D62FC72FFC011281058102950F700E94DC
:100B5000870D8823B9F01123A9F08C2F807F803472
:100B600021F080E28D0F883068F08091990282FD3B
:100B700009C082E00E94330E0E94870D91E0D82EBA
:100B8000D92601C0D12CCC2EC2948FE0C8228C2D46
:100B900090E08C30910508F0CFC1FC01E65CFF4F7E
:100BA0000C9435288C2F807FCF70882311F0C2954C
:100BB000C07F112399F0CC2309F4AAC180E28D0FE4
:100BC000883010F0D11104C08C2F0E94910D03C009
:100BD0008C2F0E94A40D0E94D30D9AC18D2F0E94CC
:100BE0003505CC2309F4A8C180E28D0F883038F197
:100BF000DD2329F18C2F0E94AA0D24C08C2F807F29
:100C0000CF70803211F0C295C07FDD2319F0D13052
:100C1000A1F13DC08091990282FF17C0112349F0D4
:100C2000CC2329F08C2F0E94910D0E94D30D80E0DF
:100C300070C180E00E943505CC2309F47DC18C2F62
:100C40000E94970D0E94D30D77C1112371F00023EC
:100C500041F0013031F40E94B40D8C2B0E94BC0D88
:100C60006BC10E94B40D8C2B1DC0002319F0013004
:100C700009F462C10E94C90D25C0112321F006307C
:100C800008F05AC10EC0053008F056C11BC0112330
:100C900061F0002331F0F701858180FF39C18F7049
:100CA00085838C2F0E94890547C1002359F0D933D1
:100CB00009F03FC1FFEF07EE13E0F1500040104094
:100CC000E1F735C18C2F0E94900536C18C2F869597
:100CD0008695837019F0813061F02EC1112321F0C7
:100CE0008D2F9C2F937002C080E090E00E94621FC5
:100CF0002BC1112321F08D2F9C2F937002C080E017
:100D000090E00E94781F20C18D2F112319F00E94BE
:100D1000E31302C00E943E140E94B51415C18C2F2B
:100D2000837009F047C011110BC12D2F2295269514
:100D30002770220F220F6D2F6F70862F90E0A0E09A
:100D4000B0E0022E04C0880F991FAA1FBB1F0A948F
:100D5000D2F7D4FF10C04FE050E060E070E004C074
:100D6000440F551F661F771F2A95D2F7409550955F
:100D70006095709503C040E050E0BA01C695C695F5
:100D8000C3708A019B01082B192B2A2B3B2BC9010D
:100D9000B801C23049F058F4C13019F00E94A608D9
:100DA000CFC00E949408CCC00E94B808C9C00E945D
:100DB0009208C6C0112319F08C2F817001C086954E
:100DC000882309F4BDC02D2F229526952770220F68
:100DD000220F6D2F6F70862F90E0A0E0B0E0022E02
:100DE00004C0880F991FAA1FBB1F0A94D2F7D4FF13
:100DF00010C04FE050E060E070E004C0440F551FA9
:100E0000661F771F2A95D2F740955095609570958B
:100E100003C040E050E0BA01C695C695C3708A0190
:100E20009B01082B192B2A2B3B2BC901B801C2307F
:100E300049F058F4C13019F00E946B0981C00E943A
:100E400059097EC00E947D097BC00E94CC0878C0F1
:100E5000CF70112339F08C2F0E94F2088D2F0E9441
:100E600089056EC08D2F0E9490058C2F0E9413095A
:100E700067C0D23F21F128F4D03F41F0D13FC1F00B
:100E800043C0D33F19F1D43F79F03EC0112341F064
:100E9000053008F051C08C2F8F710E9438094CC06A
:100EA000063008F049C0F7CF8091990282FF18C040
:100EB000112339F08C2F8F710E94F2083DC011234D
:100EC000C9F38C2F8F710E94130936C0112329F0AA
:100ED0008C2F8F710E94DD082FC00E94D8082CC073
:100EE000112349F0CF718C2F0E94F20863E08C2F00
:100EF0000E94180E21C081E00E94330E0230E0F003
:100F000082E00E94330E18C0112331F0002391F2C9
:100F10008D2F0E94DF0410C0002399F2D93349F4C9
:100F20001FEF27EE33E0115020403040E1F700C0C2
:100F300000008D2F0E94350588EF8C0D843020F441
:100F40000E942B1F0E947404DD20C9F00E94830DB3
:100F500080FD15C0F70112820E947D0D0E94F208EB
:100F6000C7010E94E0070E947D0DDF91CF911F9184
:100F70000F91FF90EF90DF90CF900C941309DF91C9
:100F8000CF911F910F91FF90EF90DF90CF90089538
:100F90000F931F93CF93DF93EC01688179818A814E
:100FA0000E94390A8C010E948F090E948008B801B2
:100FB000CE010E949705DF91CF911F910F91089567
:100FC000CF93DF93EC01988189812B813C81232B86
:100FD00031F08F3F31F481E09F3F19F403C081E08D
:100FE00001C080E080FD1DC0CE010E9494038111EC
:100FF00010C00E94870D8823A1F08A81882389F080
:101000008091990282FD0DC082E0DF91CF910C9416
:10101000330ECE010E94C807CE01DF91CF910C9410
:101020007503DF91CF910895882321F00E94A40DCC
:101030000C94D30D0895882321F00E94AA0D0C94DE
:10104000D30D089580E090E00E94621F80E090E060
:101050000E94781F0E94B10D0E94D30D0E94F415CA
:101060000C94B51480910201909103010E943A20E2
:101070000C9422080E94A10D0C94320892959F7046
:10108000963079F010F4925001C09A50923068F482
:10109000803F69F018F4883E40F409C0843F29F489
:1010A00006C0883E20F0813F11F080E0089581E085
:1010B0000895FC01808191810E942E0A0E943E08C1
:1010C0000895CF93DF9300D000D01F92CDB7DEB745
:1010D0000F900F900F900F900F90DF91CF91089588
:1010E000CF93DF9300D000D000D0CDB7DEB72696E7
:1010F0000FB6F894DEBF0FBECDBFDF91CF9108953C
:10110000089508950C9481080C9482080E94840824
:101110006093C1017093C2018093C3019093C40195
:101120000C9422080C9486080F931F930091C10120
:101130001091C2012091C3013091C401602B712B29
:10114000822B932B1F910F910C9486080F931F9362
:101150000091C1011091C2012091C3013091C401DD
:1011600060237123822393231F910F910C9486088F
:101170000F931F930091C1011091C2012091C301EF
:101180003091C40160277127822793271F910F9107
:101190000C9486080C9481080E94CA086093BD01D3
:1011A0007093BE018093BF019093C0010C942208FC
:1011B00060E070E0CB010C94CC080F931F9341E0EA
:1011C00050E060E070E08A019B0104C0000F111F35
:1011D000221F331F8A95D2F7C901B8011F910F91C1
:1011E0000C94CC080F931F9341E050E060E070E056
:1011F00004C0440F551F661F771F8A95D2F7809150
:10120000BD019091BE01A091BF01B091C0018A01C2
:101210009B01082B192B2A2B3B2BC901B8011F91CD
:101220000F910C94CC080F931F9341E050E060E0C5
:1012300070E004C0440F551F661F771F8A95D2F7D0
:1012400040955095609570958091BD019091BE013B
:10125000A091BF01B091C0018A019B01082319230D
:101260002A233B23C901B8011F910F910C94CC088C
:101270000F931F9341E050E060E070E004C0440F22
:10128000551F661F771F8A95D2F78091BD019091F7
:10129000BE01A091BF01B091C0018A019B01082746
:1012A00019272A273B27C901B8011F910F910C94D8
:1012B000CC080F931F930091BD011091BE012091A6
:1012C000BF013091C001602B712B822B932B1F919A
:1012D0000F910C94CC080F931F930091BD011091B6
:1012E000BE012091BF013091C00160237123822390
:1012F00093231F910F910C94CC080F931F9300918F
:10130000BD011091BE012091BF013091C001602745
:101310007127822793271F910F910C94CC08089571
:10132000362F292F220F920F890F982F9770A1E047
:1013300001C0AA0F9A95EAF786958695869590E062
:1013400065E070E00E94EE27FC01E854FE4F40E0AB
:1013500050E0632F70E090819B01042E02C036950F
:1013600027950A94E2F72170219529272A23292716
:1013700021934F5F5F4F4530510569F70895292F3D
:10138000220F920F890FA82FA770869586958695B4
:1013900090E065E070E00E94EE27BC0140E050E084
:1013A00080E0FB01E40FF51FE854FE4F208130E0A0
:1013B0000A2E02C0369527950A94E2F7217033274A
:1013C000042E01C0220F0A94EAF7822B4F5F5F4F71
:1013D0004530510531F70895BF92CF92DF92EF92D9
:1013E000FF920F931F93CF93DF938C01C090BD01A9
:1013F000D090BE01E090BF01F090C0018091C1018A
:101400009091C201A091C301B091C401C82AD92A08
:10141000EA2AFB2ACFE1D0E0D701C6010C2E04C096
:10142000B695A795979587950A94D2F780FD04C045
:10143000219790F7B12C07C0BC2EB8018C2F0E94C9
:1014400027110197A9F38B2DDF91CF911F910F9158
:10145000FF90EF90DF90CF90BF900895CF93DF93F0
:10146000EC010E94EC09BE010E942711DF91CF918F
:1014700008951F93CF93DF93EB019091B7019923C8
:1014800021F0CB010E942E0A13C0882349F0CB0122
:101490000E94EC09182F682FCE010E94900904C009
:1014A000CB010E94BF09182FBE01812F0E94271176
:1014B000DF91CF911F910895CF93DF93C091C50124
:1014C0008091C601C817A1F0D0E0CE0166E070E0BF
:1014D0000E94EE27FC01E953FE4F40815181628159
:1014E0007381848195810E9470082196C770E8CF2E
:1014F000DF91CF9108954091F7015091F8016091EB
:10150000F9017091FA018091FB019091FC010C941A
:101510007008FF920F931F93CF93DF938091FC018C
:1015200082958F7009F062C08091F901882309F4D7
:101530005DC02091C501F090C6011091F7010091A6
:10154000F801A091FA01B091FB0181E01F3F09F081
:1015500080E0C0910001D0910101482F2F1509F4BE
:1015600045C0109721F00F3F21F080E003C081E0DB
:1015700001C0842F30E080FD35C0C90166E070E015
:101580000E94EE27FC01E953FE4F818180132AC09F
:101590008081811327C08281811124C0838194813D
:1015A0008A1B9B0B8C179D07E8F48091FC018F70C0
:1015B00080618093FC01C90166E070E00E94EE2723
:1015C000FC01E453FE4F90819F709061908387EF00
:1015D00091E00E94E007DF91CF911F910F91FF9062
:1015E0000C945C0A2F5F3F4F2770B8CFDF91CF91EB
:1015F0001F910F91FF9008959F92AF92BF92CF924B
:10160000DF92EF92FF920F931F93CF93DF93CDB7AB
:10161000DEB761970FB6F894DEBF0FBECDBF8C0169
:1016200085E0F801DE011D9601900D928A95E1F7A3
:10163000F801E2809091F7013091F8016091FA0190
:101640007091FB016115710531F03F3F31F481E08C
:101650009F3F19F403C081E001C080E0F82FF170D2
:101660009F2E80FD47C1F80140812181A380B48075
:1016700087EFC82E81E0D82EF090F901F501E61B26
:10168000F70B6091000170910101FF2009F4DCC0AB
:101690008091FC01582F507FE617F70708F096C09D
:1016A000511155C0231313C0491311C0FE2CE11072
:1016B0000EC08F7080618093FC010E947B0AC6017E
:1016C0000E94E0078091FC01F801858350C1AB289E
:1016D00031F02F3F31F481E04F3F19F403C081E036
:1016E00001C080E080FD03C081E08E2502C080E063
:1016F00090E0F82FF170FF2E80FF1FC0E091C50130
:101700003091C601E31709F410C1F0E0CF0166E0A3
:1017100070E00E94EE27DC01A953BE4F11968C9118
:101720001197281307C08C91481304C012968C910E
:10173000E81203C03196E770E5CFFE2CEE2009F4E5
:1017400016C18091FC0181608093FC0154C0231379
:1017500006C0491304C0E11002C0F80199C0C801D5
:101760000E945908882361F1EE2051F12091FC017B
:10177000822F82958F7090E0029774F08091F7012C
:101780009091F80198878F831986BB86AA862C874B
:10179000CE0107960E94E00786E0F801A7EFB1E0CE
:1017A00001900D928A95E1F70E94890A0E947B0AB6
:1017B0000AC0231711F1C8010E94590881112CC0D9
:1017C000C8010E94E007FF24F394D1C05111F1CF6A
:1017D0007A2DB98AA88A522F6E2D89890E946108B4
:1017E00087EF91E00E94E00786E0F60111928A956A
:1017F000E9F70E947B0AF12CBAC04913DCCFE11053
:10180000DACFF8018583C8010E94E00786E0F6017F
:1018100011928A95E9F7ABC0EE2091F22091FC017C
:10182000822F82958F7090E002970CF4B5CF809153
:10183000F7019091F8019A8389831B82BD82AC8263
:101840002E83CE010196A6CFE617F70708F044C015
:10185000FE2CEE2009F4B4CF231330C049132EC060
:101860002091FC0120FD21C0822F82958F70482F8E
:1018700050E041155105C9F0F80125834F3051055D
:1018800041F08F5F982F9295907F822F8F70892BD8
:101890008583C8010E94E00786E0F801A7EFB1E068
:1018A00001900D928A95E1F73DC086E0F801A7EF1F
:1018B000B1E001900D928A95E1F759C0C8010E94EC
:1018C0005908811169CF8091FC0181608093FC01EE
:1018D000C8010E94E0074BC07A2DB98AA88A522F0E
:1018E0006E2D89890E94610886E0F60111928A9521
:1018F000E9F718C0EE2009F463CFC8010E94590827
:10190000F82E882309F45CCF86E0F801A7EFB1E058
:1019100001900D928A95E1F787EF91E00E94D9043A
:101920000E94890A0E947B0A22C04D872E878D85DE
:101930009E850E942E0A292F22952F70223028F48E
:101940009F7039F0811105C00BC0243028F49F70BE
:1019500049F4805E883020F0C8010E94E0079F2C87
:10196000F92C05C0F8019581907F99F7F9CF8F2D5B
:1019700061960FB6F894DEBF0FBECDBFDF91CF9159
:101980001F910F91FF90EF90DF90CF90BF90AF909D
:101990009F900895CF93DF93CDB7DEB72C970FB606
:1019A000F894DEBF0FBECDBF4F83588769877A8713
:1019B0008B879C87CE0107960E94FC0A8823D1F072
:1019C0009F8188852A853B85232B31F08F3F31F419
:1019D00081E09F3F19F403C081E001C080E080FDF9
:1019E0006FC04F81588569857A858B859C850E945B
:1019F000700866C086E0FE013796DE011196019000
:101A00000D928A95E1F7FF81E8856A857B856115EE
:101A1000710531F0EF3F31F481E0FF3F19F403C06D
:101A200081E001C080E080FD4BC08091C60190E064
:101A30009C012F5F3F4F277033274091C50150E035
:101A40002417350709F443C0F983EA837D836C8347
:101A500066E070E00E94EE27DC01A953BE4F96E0DD
:101A6000FE01319601900D929A95E1F72093C601FF
:101A70000E945C0A25C090E066E070E00E94EE27BC
:101A800089539E4F0E94FC0A882371F18091C50101
:101A900090E066E070E00E94EE27FC01E953FE4F03
:101AA0004081518162817381848195810E94700897
:101AB0008091C50190E00196877099278093C501B8
:101AC0008091C5019091C6018913D5CF0DC00E94A8
:101AD0003A081092C6011092C501E7EFF1E086E0E6
:101AE000DF011D928A95E9F72C960FB6F894DEBFB8
:101AF0000FBECDBFDF91CF91089580911D028595D6
:101B000085958595089580911D028770089590911F
:101B10001D02977081E009F480E0089580914002F1
:101B2000089590914002892B8093400208958095FA
:101B3000909140028923809340020895809340024F
:101B4000089510924002089590913F02892B80934E
:101B50003F020895809590913F02892380933F0230
:101B6000089510923F02089580911E0208950895ED
:101B70000C94B70D0C94B80D9091990292FD08C089
:101B800090911E02981721F080931E020C94BA0DBA
:101B9000089580911E02882329F010921E0280E091
:101BA0000C94BA0D0895CF93DF93E0910201F09168
:101BB0000301809140028083E0910201F0910301D2
:101BC000908180913F02892B808380911E0288231F
:101BD00081F0E0910201F09103019081892B8083D3
:101BE00080910201909103010E948E1F81110E9439
:101BF000C90DC0910201D091030140E250E06DEFA8
:101C000071E0CE010E945428892B69F080E2FE0128
:101C1000ADEFB1E001900D928A95E1F7CE01DF9131
:101C2000CF910C943A1FDF91CF9108950C94B70D8A
:101C30009091990292FD10C0982F990F990F990FCA
:101C4000692B60931D020E94F20880911D02859508
:101C5000859585950C94160E0C94F20810921D0231
:101C600080E00C94160E20911D02809582238093B3
:101C70001D02982F977099F430E0482F082E000C21
:101C8000550B2417350759F09091990292FD07C022
:101C90008595859585950E9413090C942E0E0895BF
:101CA0009091990292FB222720F9281769F080FB76
:101CB00092F99093990280919802909199020E94D2
:101CC000980E82E00C94330E08958091990282FB65
:101CD000882780F991E089270C94500E81E00C94BC
:101CE000500E80E00C94500E80E090E00E946F282F
:101CF00021E0893E9E4F09F020E0822F089582E086
:101D000090E00C94612883E090E00C946128CF93DC
:101D100084E090E00E946128C82F82E290E00E9457
:101D200061282C2F30E0A901582BCA01CF910895CA
:101D3000CF93C92F682F84E090E00E9475286C2F04
:101D400082E290E0CF910C947528AB01BC018FE04A
:101D500090E00C948728AB01BC0183E190E00C94E7
:101D6000872860E070E0CB010C94AB0E60E070E07F
:101D7000CB010E94A50E0C94B10E69EE7EEF80E0BF
:101D800090E00E94932860E082E090E00E94752835
:101D900060E083E090E00E9475281092C1011092EB
:101DA000C2011092C3011092C40160E084E090E08F
:101DB0000E94752860E082E290E00E94752860E051
:101DC00085E090E00E94752860E086E090E00E9447
:101DD00075286FEF87E090E00E94752840E050E0A2
:101DE000BA0188E090E00E94872860E08DE090E0F2
:101DF0000E94752840E050E0BA0188E190E00E941E
:101E0000872860E087E190E00E94752840E050E07C
:101E1000BA018CE190E00E94872860E070E080E2E7
:101E200090E00E94932840E050E0BA0188E190E001
:101E30000E9487280C94B60E0C94BD0E682F8EE07D
:101E400090E00C9475280E94F520609347027093EF
:101E500048028093490290934A0260934302709330
:101E600044028093450290934602089581E00895CC
:101E70000C94360F08950C943A0F0C943A0F0C946E
:101E80003D0F0C943A0F0C94410F0C943A0F83E0E1
:101E900092E10E94211F0E94450F0C94430F0E9463
:101EA0003B0F0C943A0F0E9406120E9473040C948C
:101EB000211C0E94E0200E94CC120E94530F0E941D
:101EC000391A0C943F0F8F929F92AF92BF92CF928C
:101ED000DF92EF92FF920F931F93CF93DF93CDB7D3
:101EE000DEB72A970FB6F894DEBF0FBECDBF0E94B3
:101EF000DB12982E81110E94230F81E4A82E82E02C
:101F0000B82E00E010E0802E802F0E942A12D82EDA
:101F1000F501C1905F01C826B1F40F5F1F4F023079
:101F2000110589F78FEF89838A831B820E94E9203C
:101F30008160782F9D838C8349815A816B818D814B
:101F40000E948F042FC080914B0281FD0E943012AD
:101F5000E12CFF24F3948C2D8F21F1F00E94380F97
:101F6000882399F0EE828F82DF2081E009F480E0FF
:101F700088870E94E9208160782F9A8789874E811F
:101F80005F8168858A850E948F04F801EF5BFD4FB1
:101F90008081F826F08206C0E394FF0CF3E0EF1294
:101FA000DACFBBCF81E0911001C080E02A960FB656
:101FB000F894DEBF0FBECDBFDF91CF911F910F917F
:101FC000FF90EF90DF90CF90BF90AF909F908F9059
:101FD00008950E94630F0E946C1A0E94D3140C94FF
:101FE0008404CF93DF930E942C11EC01811521E52D
:101FF000920708F045C0811530E5930708F094C0BA
:10200000883E910528F5803E910508F001C1883A87
:10201000910570F4853A910508F07CC081309105F6
:1020200009F475C008F4F1C0049708F0F1C0EDC0E0
:102030008F3B910508F0E9C0C85AD0E0CC0FDD1FF6
:10204000C45ADE4F0990D881C02DCE019464E1C0FE
:10205000811540E2940758F4811551E0950708F086
:10206000D7C08D3E910508F4D0C09065D2C0C1158F
:1020700080E4D80708F4C9C0DF70CE01906AC9C0F7
:10208000811525E59207A8F4811534E5930708F03A
:102090009EC0811543E5940708F081C0811552E583
:1020A000950708F064C0D82FCC27CE01816F906AC5
:1020B000B0C0C11589E5D807A0F4C11528E5D2073D
:1020C00008F08BC0C11536E5D30708F09EC08C2FF1
:1020D0000E94C0118F7190E0D82FCC27CE01906262
:1020E00098C0C1154AE5D40708F47DC0CE019056CA
:1020F0008115904208F089C08D2F8F710E94C01108
:10210000DD27D0628F71AE01582BCA0182C081E0F9
:1021100090E07FC0C55AD0E0C657DE4F8881C82FF7
:10212000D0E0CE01906475C0F4E096958795FA955D
:10213000E1F7282F23703C2F337081E090E002C03C
:10214000880F991F3A95E2F79C68AC01522B9C2F9F
:102150009F7096959695892F90E0EC01A5E0CC0FA5
:10216000DD1FAA95E1F7CA018C2B9D2B52C083700D
:10217000992721E030E002C0220F331F8A95E2F751
:102180009C2F96959695C92FD0E075E0CC0FDD1F5A
:102190007A95E1F7C22BD32BCE019C683AC08370AD
:1021A000992721E030E002C0220F331F8A95E2F721
:1021B0009C2F96959695C92FD0E065E0CC0FDD1F3A
:1021C0006A95E1F7C22BD32BCE019A6822C0D82F93
:1021D000CC27CE01846F906A1CC0DC2FCC27CE01A7
:1021E000806F906A16C08C2F8F700E94C01194E08F
:1021F000D695C7959A95E1F7CF70D0E0DC2FCC2724
:10220000D0699E01282BC90104C080E090E001C084
:10221000CE01DF91CF910895382F262F872F90E0A0
:1022200063E070E00E94EE27FC01832F90E066E0FF
:1022300070E00E94EE278E0F9F1FFC01E20FF11D40
:10224000EE0FFF1FE056FF4F8591949108950E9475
:102250000C110E94F10F08958238910569F1B0F4D4
:102260008133910509F46DC048F48932910509F470
:1022700063C08A32910509F469C0089585339105D8
:1022800009F455C089339105B9F00895833E91054D
:1022900069F138F4803E9105B1F0823E910509F173
:1022A0000895863E9105A9F1873E9105B9F1843ED6
:1022B000910509F064C023C02091980220FD4FC011
:1022C00021FD4DC008958091980280FD44C0809109
:1022D000990280FF44C08091980284FD42C083EE41
:1022E0004DC08091980282FF38C0F5CF809198024E
:1022F00082FD33C08091990280FD31C0ECCF809186
:10230000990281FF32C08091980284FD2AC087EE35
:1023100035C08091980283FF26C0F5CF8091980246
:1023200083FD21C08091990281FD1FC0ECCF809177
:10233000980285FD1CC01DC08091980285FD19C0C2
:1023400016C08091980286FD16C017C08091980231
:1023500086FD13C010C089E311C082EE0FC080EE6D
:102360000DC080E00BC086EE09C084EE07C089E294
:1023700005C085E303C08AE201C081E390E00895CF
:102380009091980292FF0DC0282F2871283019F4DF
:10239000877F846006C0282F2471243011F48B7F3E
:1023A000886093FF0DC0282F2871283119F4877E8B
:1023B000846106C0282F2471243111F48B7E88613A
:1023C0002091990220FF0DC0382F3871383019F450
:1023D000877F816006C0382F3171313011F48E7FD4
:1023E000886021FF0DC0282F2871283119F4877EBD
:1023F000816106C0282F2171213111F48E7E886100
:1024000094FD877E089580E0089508950E94740EDB
:10241000811102C00E941C0F0E947F0E80934B020C
:102420000E94870E90939902809398020E94051251
:102430000E94830E682F70E080E090E00E94920876
:102440006091BD017091BE018091BF019091C0016A
:102450000C94CA08E82FF0E0E456FD4F80810895FF
:10246000089580EA8A95F1F7089500C008950C94C4
:10247000311208950C9439120C943A120C943912BA
:102480000C943E12F894E82FE295EF70F0E031A141
:10249000282F2F7081E090E001C0880F2A95EAF77D
:1024A000982F9095932391A392A1892B82A378943E
:1024B000089583E30E94421284E30E94421280E363
:1024C0000E94421281E30E94421282E30C94421263
:1024D000CF92DF92EF92FF920F931F93CF93DF93F0
:1024E0008C01C62FD0E0CE0180579E4F7C01FC01AD
:1024F00090819F3F09F447C0D62EF894E92FE295CA
:10250000EF70F0E081A19F7021E030E001C0220F68
:102510009A95EAF7822B81A382A12095282322A3F2
:1025200078940E943512EDE8F1E040E951E031E0A5
:10253000C12C21912F3F89F0A22FA295AF70B0E05E
:1025400090968C9190E02F7002C0959587952A9572
:10255000E2F780FD02C0832F01C080E0C82A330F5C
:102560004E175F0731F7F70180818F3F11F00E940E
:10257000421261E0C11001C060E08D2D0E9437124F
:10258000C00FD11FC882DF91CF911F910F91FF9093
:10259000EF90DF90CF9008950E94591210929D0203
:1025A00010929C0210929B0210929A0282E00E946A
:1025B00013130C9480031F93CF93DF9300D0CDB7F8
:1025C000DEB71A82198260E0CE0101960E9468127D
:1025D00061E0CE0101960E94681242E050E0BE0127
:1025E0006F5F7F4F8AE992E00E94542811E00097C4
:1025F00009F410E0892B31F089819A8190939B0234
:1026000080939A02212F42E06CE972E08AE992E01D
:102610000E9414130E948203812F0F900F90DF916C
:10262000CF911F9108950895FF920F931F93CF9319
:10263000DF938C01F62ED72FC42F222349F081E09F
:1026400080934E020E94E92090934D0280934C02A9
:1026500080914E028823C1F080914C0290914D02EE
:102660000E940121059780F0EF2DFD2FD8014C2FFE
:1026700050E0CD01801B910B841795071CF48D91C0
:102680008193F7CF10924E02DF91CF911F910F915E
:10269000FF9008950E94EC220E94590F0C94F8229A
:1026A0000E94FC220E94E90F0C9416230E948720AE
:1026B0000E94D3220E94470F0E944A130E94501387
:1026C0000E944F0FFBCF8091550280FF06C06091A2
:1026D000090170E0660F771F2CC081FF08C0609170
:1026E000090170E0660F771F660F771F22C082FF17
:1026F00009C06091090170E043E0660F771F4A95B9
:10270000E1F717C0609154026623D1F020910801CF
:10271000621778F78091090190E070E033E0880F4C
:10272000991F3A95E1F70E94EE27622F70E00E9410
:1027300021286038710540F46115710519F406C04F
:1027400068E070E0862F08958FE7089581E008958E
:102750008091550280FF08C06091050170E0759579
:1027600067957595679523C081FF06C06091050147
:1027700070E0759567951BC082FF04C060910501EC
:1027800070E012C0609153026623A9F02091040109
:102790006217A0F78091050170E090E00E94EE279B
:1027A000622F70E00E9421286038710540F46115A5
:1027B000710519F406C061E070E0862F08958FE777
:1027C000089581E008958D3E21F40E946313819560
:1027D00004C08E3E29F40E94631380935902089529
:1027E0008F3E21F40E946313819504C0803F29F439
:1027F0000E946313809358020895893F19F40E9440
:10280000A81305C08A3F31F40E94A81381958093D4
:102810005A0208958B3F21F40E94A813819504C0A9
:102820008C3F29F40E94A81380935B0208959FE0D7
:10283000980F983078F421E030E0A90102C0440FED
:10284000551F9A95E2F7CA0190915702892B809300
:10285000570208958D3F21F48091550281600BC08D
:102860008E3F21F480915502826005C08F3F29F48C
:102870008091550284608093550208958D3E39F40D
:102880009091590297FF35C01092590259C08E3E5F
:1028900029F4909159021916BCF32BC0909158025B
:1028A0008F3E29F497FF25C01092580249C0803FFF
:1028B00019F41916CCF31DC090915A02893F29F4DE
:1028C0001916BCF410925A023BC08A3F19F497FFC4
:1028D00010C0F8CF8B3F39F490915B0297FF09C08D
:1028E00010925B022DC08C3F21F490915B0219166F
:1028F000BCF39FE0980F983080F421E030E0A9010C
:1029000002C0440F551F9A95E2F7CA018095909135
:10291000570289238093570213C08D3F21F4809181
:1029200055028E7F0BC08E3F21F4809155028D7F22
:1029300005C08F3F29F4809155028B7F809355020B
:1029400080915802811106C080915902811102C004
:102950001092540280915A02811106C080915B024C
:10296000811102C01092530208950E94E920209123
:102970005802211104C020915902222321F0909382
:1029800052028093510220915A02211104C02091D9
:102990005B02222321F09093500280934F0286E540
:1029A00092E00C94541FEF92FF920F931F93CF93DA
:1029B000DF9300D000D000D0CDB7DEB786E0E6E5EB
:1029C000F2E0DE01119601900D928A95E1F7E09018
:1029D0005802F090590200915A0210915B02109235
:1029E00058021092590210925A0210925B02E110A2
:1029F00003C0FF2009F464C08091510290915202FB
:102A00000E940121FC0120915402222339F080917F
:102A10000A0190E08E179F0760F052C080910B0171
:102A200090E06AE070E00E94EE278E179F0718F092
:102A300047C02F3F19F02F5F20935402EE2061F022
:102A40000E946313682F1E1414F08FEF01C081E001
:102A50000E94E52780935802FF2061F00E946313D3
:102A6000682F1F1414F08FEF01C081E00E94E5274A
:102A70008093590280915802882311F120915902C4
:102A80002223F1F0082E000C990B65EB70E00E94F8
:102A9000EE27992319F09093580203C081E08093A8
:102AA0005802822F220F990B65EB70E00E94EE27EF
:102AB000992319F09093590203C081E08093590241
:102AC000011103C0112309F464C080914F02909159
:102AD00050020E940121FC0120915302222339F06F
:102AE0008091060190E08E179F0760F052C08091A0
:102AF000070190E06AE070E00E94EE278E179F07C2
:102B000018F047C02F3F19F02F5F20935302002386
:102B100061F00E94A813682F101614F08FEF01C007
:102B200081E00E94E52780935A02112361F00E9400
:102B3000A813682F111614F08FEF01C081E00E94D6
:102B4000E52780935B0280915A02882311F120913E
:102B50005B022223F1F0082E000C990B65EB70E06C
:102B60000E94EE27992319F090935A0203C081E046
:102B700080935A02822F220F990B65EB70E00E941E
:102B8000EE27992319F090935B0203C081E08093B4
:102B90005B028091580281110BC080915902811112
:102BA00007C080915A02811103C080915B0281119C
:102BB0000E94B514EB82FC820D831E8386E0FE0129
:102BC0003196A6E5B2E001900D928A95E1F726963E
:102BD0000FB6F894DEBF0FBECDBFDF91CF911F912E
:102BE0000F91FF90EF900895E6E5F2E086E0DF01B7
:102BF0001D928A95E9F71092540210925302109296
:102C000055020895EF92FF920F931F93CF93DF9396
:102C1000E82F71110AC0442321F0F0E0E757FD4F7F
:102C2000E4916E2F7E2F8E2F6CC0C62FD0E0072F21
:102C300010E0282F30E0442329F0F901E757FD4F39
:102C4000249130E0CE0166E070E00E94EE27EE2491
:102C5000EA94F12CB7010E940D28DB01CC0FDD1F97
:102C6000CB016BEA7FEF0E94EE278C0F9D1FC82FD0
:102C7000CC0FC80FC701801B910BB9010E94EE2732
:102C8000E92F492FD0E0CE01B8010E94EE27692F2D
:102C900070E0C701861B970BB9010E94EE27F92F40
:102CA000C7018C1B9D0BB8010E94EE27692F70E0B5
:102CB000C701861B970BB9010E94EE27A230B10510
:102CC00091F038F4109759F01197C1F48E2F7F2F9F
:102CD0000CC0A430B10579F050F0169779F4722F3A
:102CE000842FE92F0DC0892F7E2FE22F09C0822F5C
:102CF0007E2FEF2F05C0822F792F02C0722F8F2FCA
:102D00006E2FDF91CF911F910F91FF90EF9008955B
:102D100041E00E940216089508950E9488160895C1
:102D2000CF93DF93762FE901682F842F0E948D16B1
:102D3000798368838A83DF91CF91089580919E0281
:102D4000282F269530E02115310519F48170826015
:102D500005C02232310524F08170826480939E0286
:102D6000089588E090E00C946928CF92DF92EF926A
:102D7000FF926B017C010E949E16B701A60188E0BC
:102D800090E0FF90EF90DF90CF900C948728EEE9D1
:102D9000F2E083E0808311828FEF82838383148249
:102DA00060817181828193810C94B51680919E021D
:102DB00080FF02C08695089580E008959091A20258
:102DC000933018F49F5F9093A202882351F0609192
:102DD0009E0270919F028091A0029091A1020C949A
:102DE000B516089581E00C94DE169091A202992305
:102DF00019F091509093A202882351F060919E02A5
:102E000070919F028091A0029091A1020C94B5163E
:102E1000089581E00C94F51670E00C94CE1B30916F
:102E20000F0180919E0280FF0CC080910E0190E006
:102E300063E070E00E94EE27632F8D559D4F0C9448
:102E40000C172091100140911101241770F7822F67
:102E500090E063E070E00E94EE27FC01ED55FD4F2D
:102E60001182108212822F5FF0CFA82FB62F80918F
:102E70009E0280FF16C0209110013091110123178E
:102E800070F4822F90E063E070E00E94EE27FC0176
:102E9000ED55FD4FA183B08342832F5FF0CF0C949B
:102EA0000F170895CF93DF9300D01F92CDB7DEB7F1
:102EB00090919E0290FF0AC09E012F5F3F4F0E949B
:102EC00090164B8169818A810E9435170F900F906F
:102ED0000F90DF91CF910895CF93DF93EC01EC81B8
:102EE000F0E0EC57FE4F4491EEE9F2E0628181811F
:102EF0000E9452178C818F5F8C83DF91CF91089550
:102F0000CF93DF93EC01EEE9F2E0438162818C81A3
:102F10000E9452178C818F5F8C83DF91CF9108952F
:102F2000AF92BF92CF92DF92EF92FF920F931F93D7
:102F3000CF93DF9300D01F92CDB7DEB7182FF62EB8
:102F4000042FE22E90919E0290FF6EC0E92FE6952D
:102F5000AE2FB0E0AE56BE4F8C91809365029E7F3F
:102F6000923061F49E012F5F3F4F812F0E94901697
:102F70004B8169818A810E94351744C0823019F4DF
:102F80000091A1023FC0863019F410919F023AC00F
:102F90008930D9F38831B1F5E8514E2F4170D42EE4
:102FA000E695F0E0EC57FD4FA590B490C12CBB2402
:102FB00040911201C41620F52C2D30E0C501B90155
:102FC0000E94EE27642F70E00E940D28E12FD1109F
:102FD00002C0E60F01C0E61B80911001A901480F55
:102FE000511DCA0163E070E00E94EE279C012D553F
:102FF0003D4F402F6F2D8E2F0E949016C394D8CF37
:103000000E940F1710939F02F092A0020093A1025A
:10301000EE2051F060919E0270919F028091A0027B
:103020009091A1020E94B5160F900F900F90DF9122
:10303000CF911F910F91FF90EF90DF90CF90BF90B5
:10304000AF900895EEE9F2E09181282F43816281EB
:103050008AE0890F0C94901781E00C942218EEE915
:10306000F2E09181282F4381628186EF890F0C94D1
:10307000901781E00C942F18EEE9F2E0628121E1D3
:10308000620F08F46FEF282F438181810C94901711
:1030900081E00C943C18EEE9F2E0628121E1621BD0
:1030A00008F460E0282F438181810C94901781E01F
:1030B0000C944B18EEE9F2E0438121E1420F08F451
:1030C0004FEF282F628181810C94901781E00C943E
:1030D0005A18EEE9F2E0438121E1421B08F440E096
:1030E000282F628181810C94901781E00C946918DB
:1030F00020E00C949017EF92FF921F93CF93DF93F1
:10310000EC0110E0EE24EA94F12C30911201131737
:1031100000F520911001812F90E0820F911D63E056
:1031200070E00E94EE27FC01ED55FD4F632F70E02B
:10313000C7010E942128812F0E94E5279C819F01C1
:103140004091A1026091A002890F0E9490161F5F1A
:10315000DCCF0E940F179A818C8190FF02C08F5F95
:1031600001C081508C83DF91CF911F91FF90EF9030
:103170000895AF92BF92CF92DF92EF92FF920F939A
:103180001F93CF93DF93FC01828180FF02C0DFEFAA
:1031900001C0D1E0C0E03AE0A32E80911201C8172F
:1031A00008F043C080911001CC2ED12C9601280F3D
:1031B000311DC90163E070E00E94EE278D559D4FDF
:1031C0007C01FC0111821082128204E010E0B12C1B
:1031D00080915D028B0D8B302CF06A2D0E94FF27B1
:1031E000892F05C087FF03C090911201890F082E17
:1031F000000C990BC816D90691F48091A10290E0B9
:10320000B8010E94EE27959587959595879597012A
:10321000482F6091A00280919F020E949016BD0EDF
:1032200001501109A9F6CF5FB8CF0E940F17809106
:103230005D02D13031F4811102C0809112018150C0
:1032400007C090E001966091120170E00E94212871
:1032500080935D02DF91CF911F910F91FF90EF90CE
:10326000DF90CF90BF90AF900895CF932091100141
:1032700030911101231770F4822F90E063E070E029
:103280000E94EE27FC01ED55FD4F11821082128243
:103290002F5FF0CFC0E060911201C61790F5EC2FC0
:1032A000F0E070E0CF010E94212890911001890F79
:1032B00020915C02022E000C330B90E063E070E082
:1032C0000E94EE27E217F307A4F020910D01022ED1
:1032D000000C330B2E173F0764F09C012D553D4F1A
:1032E0004091A1026091A00280919F020E949016DD
:1032F00006C0FC01ED55FD4F118210821282CF5F96
:10330000CACF0E940F1720910C0180915C02820F9E
:1033100080935C0290910D01920F90930D0119160C
:103320005CF4082E000C990B4091120150E04150C2
:103330005109841795071CF0219520930C01CF911A
:103340000895EEE9F2E080818E7F80836081718153
:10335000828193810E94B516109266022FEF80E75A
:1033600092E0215080409040E1F700C000000C94B2
:103370000F1760919E02669570E04BE050E083E18C
:1033800091E00E944728892B19F481E0809366021E
:103390000E94E92090935F0280935E0208959091CD
:1033A0009E0290FF35C09170811102C0926006C0EC
:1033B000823210F0926402C0880F982B90939E0284
:1033C000662351F060919E0270919F028091A0024D
:1033D0009091A1020E94B51660919E02669570E0E0
:1033E0004BE050E083E191E00E944728892B19F0DF
:1033F0001092660202C00E94B91981E080936102B6
:103400004091A1026091A00280919F020C947818D3
:103410000895682F90919E02969581E0890F8232DF
:1034200008F081E00C94CF1981E00C94091A682F00
:1034300090919E0296958FEF890F09F481E20C948A
:10344000CF1981E00C94171A61E00C94CF19EEE9C2
:10345000F2E080818160808386950C94241A8091AB
:103460009E0280FD0C94A1190C94271A60E00C9424
:10347000CF198091640281112EC00E94740E8111B7
:1034800004C00E941C0F0E94C7160E94B1166093D0
:103490009E0270939F028093A0029093A1026E7F80
:1034A00061F40E94C7160E94B11660939E02709349
:1034B0009F028093A0029093A1020E949E161092F8
:1034C000660280919E0280FF03C086950E94361A94
:1034D00081E08093640208950F931F93CF93DF934D
:1034E00080916602882309F46EC080916502E091A4
:1034F0009E02E695E81BE0936002823049F4F0E01A
:10350000E058FE4FE491CE2FD0E00CE617E132C038
:10351000863049F4F0E0E358FE4FE491CE2FD0E03E
:1035200000E817E127C0893051F4E695F0E0E6584D
:10353000FE4FE491CE2FD0E00BE718E11BC08F3097
:1035400051F4E695F0E0E958FE4FE491CE2FD0E03B
:1035500009EB18E10FC0853149F4F0E0EC58FE4F5B
:10356000E491CE2FD0E005E319E104C0C0EDD7E02F
:103570000CE816E180916102882361F010926102EB
:103580000E94E92090935F0280935E021092630292
:10359000109262020E94E920E0915E02F0915F02C7
:1035A0008E1B9F0B8F3F9F4770F4EC0FFD1FF09316
:1035B0005F02E0935E028EE592E0F801DF91CF9129
:1035C0001F910F910994DF91CF911F910F91089551
:1035D000882311F0FA0101C0FB010994CF93DF9316
:1035E000C82FD62F0E94D6168C1740F00E94D616F0
:1035F0008D1720F4DF91CF910C94141A8C2FDF914A
:10360000CF910C94241A1F93CF93DF93FB01128167
:103610001111BFC0EC010E948E0D8272CD3CFCE501
:10362000DF0709F49AC0A8F5C73CECE5DE0709F40A
:1036300076C0A8F4C43C9CE5D90709F45FC028F41F
:10364000C33CDC4509F457C054C0C53C9CE5D907D0
:1036500009F459C0C63CDC4509F45CC04AC0CA3C08
:10366000FCE5DF0709F46AC050F4C83CECE5DE076E
:1036700009F45AC0C93CDC4509F45BC03AC0CB3CF4
:103680009CE5D90709F45FC0CC3CDC4509F460C077
:1036900030C0C23DFCE5DF0709F471C088F4CF3CBF
:1036A0009CE5D90709F462C008F45CC0C03DFCE5A4
:1036B000DF0709F45EC0C13DDC4509F45DC019C0F7
:1036C000C53D9CE5D90709F460C050F4C33DFCE555
:1036D000DF0709F457C0C43DDC4509F45AC009C0EE
:1036E000C63D9CE5D90709F454C0CE35DD4509F443
:1036F00050C011E04EC00E942F1A4BC041E25AE167
:1037000064E17AE104C044E15AE161E27AE10E94B5
:10371000E81A3FC049E358E16CE278E1F8CF4CE2A7
:1037200058E169E378E1F3CF47E558E168E478E1EF
:10373000EECF48E458E167E578E1E9CF45E758E1A5
:1037400066E678E1E4CF46E658E165E778E1DFCF69
:1037500049E057E162EF76E1DACF42EF56E169E006
:1037600077E1D5CF81E00E94241A13C065E082E0A2
:103770000EC068E086E00BC06EE089E008C064E13E
:103780008FE005C067E185E102C061E288E10E9447
:10379000EE1A812FDF91CF911F910895529A2BB18C
:1037A0002B7F3BB134604FB7F894FC01CB0163E051
:1037B00070E00E94EE278E0F9F1FE817F90789F02F
:1037C000519168E03BB9000000C057FF2BB9550F7D
:1037D000000000C000C000C02BB900C06A9591F77E
:1037E000ECCF4FBF8FE594E00197F1F700C00000E8
:1037F0000895CF93DF9397FF0DC0FB012281222311
:1038000049F0EC010E94371CCE019F770E94AA1C50
:103810000E94841C81E0DF91CF9108959091C202B3
:10382000923069F48A3040F490E009966AE070E0E2
:103830000E942128875A01C086500C9480050C9460
:1038400062048CE090E00E94612890E0A0E0B0E08B
:103850008093C2029093C302A093C402B093C502A6
:1038600008956091C2028CE090E00C9475280E944B
:10387000371F869581708093C7020E94371F817021
:103880008093C1028091C202813039F48091C702D5
:10389000882319F089E30E9480050E948E0D809391
:1038A000C6020E94A10D8091C202813071F048F0E1
:1038B000823081F0843009F586EE0E94800588E12F
:1038C0001AC082EE0E94DF0418C088E193E00E94D3
:1038D000180313C08091C102811103C083E50E94C7
:1038E000800582EE0E94DF048FE39CE90197F1F7E7
:1038F00000C0000087E50E9480058FE39CE90197E6
:10390000F1F700C0000008958091C202813059F0A3
:1039100030F0823089F08430C9F488E215C082EE3C
:103920000E94350513C08CE20E9480058091C70279
:10393000882361F089E308C082EE0E9435058091FA
:10394000C102811103C083E50E9480058091C602F7
:103950000C949E0D0F931F93CF93DF938C01CCE0BB
:10396000D0E0C8010C2E02C0969587950A94E2F724
:103970008F700E940E1C2497CC3F8FEFD80789F7D9
:10398000DF91CF911F910F9108950F931F93CF93C4
:10399000DF93EC018B01FB018281882361F00E949F
:1039A0008E0DCE01825E9C458530910520F480937A
:1039B000C2020E94311CB801CE01DF91CF911F914C
:1039C0000F910C94F91BCF93DF93EC01FB018281E3
:1039D000882309F43CC1C430FDE5DF0760F4CB3F28
:1039E0009CE5D90788F49E0122503C4524313105DD
:1039F00008F02EC109C0C236EDE5DE0729F0C63A4F
:103A0000FDE5DF0709F024C10E94870E909399021B
:103A100080939802C1318CE5D80709F4C6C008F03C
:103A200042C0C930ECE5DE0709F49BC000F5C530A3
:103A30008CE5D80709F485C078F4C330ECE5DE07DF
:103A400009F478C008F07AC0C230DC4509F0F5C04E
:103A5000809198028160EFC0C7309CE5D90709F4D6
:103A600078C008F07AC0809198028061E4C0CD30BF
:103A7000FCE5DF0709F487C058F4CB309CE5D90793
:103A800009F479C008F07BC08091980288606FC00B
:103A9000CF30FCE5DF0709F480C008F082C08091D8
:103AA0009802877FC8C0CE3F9CE5D90709F471C052
:103AB00000F5C531FCE5DF0709F485C068F4C331C2
:103AC0009CE5D90709F475C008F095C00E943A0832
:103AD000809198028F77AFC0CC3FFCE5DF07A9F15A
:103AE00008F054C0CB3FDC4509F0A7C08091990293
:103AF00040C0C230EDE5DE0709F489C058F4C115B5
:103B00008DE5D80709F45AC008F069C08091990280
:103B100082602FC0C236EDE5DE0709F47CC0C63AEC
:103B2000FDE5DF0709F481C0C330DD4509F085C03C
:103B300080E06EC08091980282607DC08091980282
:103B400016C080919802886076C080919902826048
:103B50004FC08091980280626EC08091980280640C
:103B60006AC00E943A0880919802806864C08460AC
:103B700062C081603DC0809198028E7F5CC0809160
:103B800098028D7F58C08091980216C0809199024A
:103B900018C0809199028D7F2BC0809198028F7EF2
:103BA0004AC0809198028F7D46C0809198028F7B99
:103BB00042C080919802877F8B7F3DC0809199029F
:103BC0008D7F8E7F15C08091980282FB222720F97D
:103BD00091E0922790FB82F990FB83F92CC08091B1
:103BE0009902982F909591708E7F892B90FB81F987
:103BF0008093990222C00E943A088091980287FB24
:103C0000222720F991E0922790FB87F914C081E0E8
:103C10000E941E0F12C08091980284FB222720F977
:103C200091E0922790FB84F906C080919802982F2A
:103C3000909590FB80F980939802809198029091E2
:103C400099020E94980E0E943A0880E001C081E02B
:103C5000DF91CF910895CF93DF9386319C4541F555
:103C6000EB010E948E0D982F8A81209102013091E4
:103C70000301882379F09A7A81E009F480E0809347
:103C80006702911102C069E201C065E3C9010E94A7
:103C900024200AC080916702811102C069E201C03C
:103CA00065E3C9010E942F200E94D30D80E001C06E
:103CB00081E0DF91CF9108950F931F93CF93DF930E
:103CC000C42FD22FFC0182818823C9F040936A025D
:103CD0000E94E920909369028093680280E28C0F31
:103CE000883008F057C0C77081E001C0880FCA95BE
:103CF000EAF7DF91CF911F910F910C948905809184
:103D00006A02481330C080916802909169020E9453
:103D10000121883C910538F510E21D0FCD17B9F04F
:103D200080E28C0F883040F4C77081E001C0880FBA
:103D3000CA95EAF70E949005183028F581E09D2F7A
:103D4000977001C0880F9A95EAF70E948905802F25
:103D50000E9480051830F0F4D77081E001C0880F10
:103D6000DA95EAF70AC080E28C0F883098F4C770C1
:103D700081E001C0880FCA95EAF7DF91CF911F91CA
:103D80000F910C949005802FDF91CF911F910F918F
:103D90000C948005DF91CF911F910F9108950F939F
:103DA0009C01CB01243F4CE5340731F188F4293DD7
:103DB000FCE53F07D9F02A3D4CE5340779F1283D71
:103DC0003C45A9F506E221EE41EE68ED7CE52BC00D
:103DD000263FFCE53F07E1F0A8F0273F3C4539F5D9
:103DE00007E225EE46EE67EF7CE51DC007E225EE13
:103DF00045EE69ED7CE517C006E221EE40EE64EF8A
:103E00007CE511C007E225EE44EE65EF7CE50BC0D2
:103E100006E221EE42EE66EF7CE505C008E221E015
:103E200045EE6AED7CE50E945C1E80E008C0FC0166
:103E30008281882319F010926A0201C081E00F91FB
:103E400008959093B5018093B40108959093700202
:103E500080936F020895E0916F02F09170023097A5
:103E600021F00190F081E02D099480E008950E94F6
:103E70002B1F0895E0916F02F0917002309799F036
:103E800020912A01222359F02091980227FF07C090
:103E9000DC012C9111962C93119726E02C93028033
:103EA000F381E02D09940895E0916F02F091700282
:103EB000309739F022E0DC012C930480F581E02D6D
:103EC0000994089520916D0230916E0228173907E8
:103ED00071F090936E0280936D02E0916F02F09109
:103EE0007002309721F00680F781E02D0994089543
:103EF00020916B0230916C022817390771F0909372
:103F00006C0280936B02E0916F02F0917002309727
:103F100021F00084F185E02D09940895FC0132968A
:103F200080912A01882331F08091980287FF02C096
:103F30009EE101C096E080E0915028F0219122237B
:103F4000D9F38F5FF9CF0895662351F120912A01AB
:103F50002223E9F02091980227FF19C0462F4695A9
:103F6000469546954E31E0F4677021E030E002C09E
:103F7000220F331F6A95E2F7FC01E40FF11D8281E5
:103F800090E02823392381E0232B69F409C0FC0148
:103F9000329608962191621729F0E817F907D1F7B0
:103FA00080E0089581E008959C01FC0132969FEF26
:103FB00080E04191461789F09F3F19F4411101C0FB
:103FC000982F8F5F8630A9F79F3F39F0F901E90FED
:103FD000F11D97FDFA956283089508959C012A5F6B
:103FE0003F4FFC014281461301C0128201968217A5
:103FF0009307B9F70895262F2695269526952E31F5
:1040000068F4FC01E20FF11D677021E030E001C0AF
:10401000220F6A95EAF78281282B22830895262FA2
:104020002695269526952E3170F4FC01E20FF11DA0
:10403000677021E030E001C0220F6A95EAF7209511
:10404000828128232283089520912A01222329F0A6
:104050002091980227FD0C94FB1F0C94D41F2091F3
:104060002A01222329F02091980227FD0C940F2089
:104070000C94EE1F20912A01FC013296222331F08C
:104080008091980287FF02C08EE101C086E0DF01C7
:104090001D928A95E9F7089508950C944C2083E0C9
:1040A000809371020C944D20811102C081E001C007
:1040B00082E0809371020C944D200C94542081E096
:1040C000809371020C944D200C945F2008950C9401
:1040D00066200C9467200C9466200C9466200C9447
:1040E00066200E946D200E94DB120E946B2080E0FF
:1040F0000E942A12811108C081E00E942A1291E0D8
:10410000811103C090E001C091E0892F08950895C6
:104110001F920F920FB60F9211248F939F93AF931C
:10412000BF9380917202811113C08091C802909157
:10413000C902A091CA02B091CB024196A11DB11D46
:104140008093C8029093C902A093CA02B093CB0295
:10415000BF91AF919F918F910F900FBE0F901F90C5
:1041600018958091D002843031F10E94F4031092AE
:10417000720220E488E190E00FB6F894A89580934D
:1041800060000FBE2093600083B7817F846083BF8F
:1041900083B7816083BF7894889583B78E7F83BF10
:1041A0000FB6F894A89580916000886180936000B4
:1041B000109260000FBE08950E943A080C94F80314
:1041C00082E084BD93E095BD9AEF97BD80936E0029
:1041D00008952FB7F8948091C8029091C902A091D8
:1041E000CA02B091CB022FBF08952FB7F894609107
:1041F000C8027091C9028091CA029091CB022FBF70
:1042000008959C014FB7F8948091C8029091C9021B
:10421000A091CA02B091CB024FBF821B930B0895AD
:1042200078941F920F920FB60F9211248F939F9341
:10423000AF93BF938091C8029091C902A091CA0226
:10424000B091CB020196A11DB11D8093C80290933D
:10425000C902A093CA02B093CB02BF91AF919F91C4
:104260008F910F900FBE0F901F90189581E0809353
:10427000E00080E28093D8001092C9008FE19EE4B4
:104280000197F1F700C0000087E090EBDC0180931C
:10429000D9029093DA02A093DB02B093DC029CE097
:1042A00088E10FB6F894A895809360000FBE9093B4
:1042B0006000FFCF809196020895089522E0209338
:1042C000E9002FEF3091E800215035FD06C035EDB3
:1042D0003A95F1F700002111F5CF2091E80025FF74
:1042E0000BC040E050E066E070E00E9488238091BF
:1042F000E8008E778093E8000895CF93DF932091B4
:104300002A01222339F02091980227FF03C060E29E
:1043100022E002C068E021E02093E9002FEF309115
:10432000E800215035FD06C035ED3A95F1F7000063
:104330002111F5CF2091E80025FF1DC0EC018091EF
:104340002A01811105C040E050E068E070E003C040
:1043500070E040E050E0CE010E9488238091E800A8
:104360008E778093E80080E2FE01A6E7B2E001903C
:104370000D928A95E1F7DF91CF91089580937302B2
:1043800070937502609374028091D002843001F5BD
:1043900082E08093E9008FEF9091E800815095FDD5
:1043A00006C095ED9A95F1F700008111F5CF809147
:1043B000E80085FF0DC040E050E063E070E083E777
:1043C00092E00E9488238091E8008E778093E80035
:1043D0000895BC0184E00C94BE21BC0183E00C94E0
:1043E000BE210C9464206091CC0281E0611101C077
:1043F00080E00C944F209091D00281E0943009F03D
:1044000080E06091CC020C94542042E061EC81E0A9
:104410000E948C2442E261EC82E00E948C24909104
:10442000D00281E0943009F080E06091CC020C94DD
:104430005D208091D202833009F45DC030F4813078
:1044400071F0823009F496C008958A3009F482C070
:104450008B3009F468C0893009F0A4C020C0809175
:10446000D102813A09F09EC08091E800877F809355
:10447000E8008091D5029091D602892B21F460E268
:1044800086E792E003C060E080E090E070E00E9488
:10449000D3238091E8008B778093E8000895809182
:1044A000D102813209F07EC08091D5029091D6026E
:1044B000029708F077C08091E800877F8093E8003A
:1044C0008091E80082FD05C08091D0028111F8CF73
:1044D00069C08091F200823031F48091F100813026
:1044E00011F0863021F48091F10080939602809142
:1044F000E8008B7753C08091D102813A09F052C015
:104500008091D5029091D602892B09F04BC0809101
:10451000E800877F8093E8008091E80080FFFCCF6F
:1045200080912A0136C08091D1028132D9F58091E3
:10453000D5029091D602892BA9F58091E800877F5A
:104540008093E8000E94C1248091D30280932A01C5
:104550000C943A088091D102813221F58091E800D3
:10456000877F8093E8000E94C1248091D4028093C9
:10457000970208958091D102813AA1F48091E800D8
:10458000877F8093E8008091E80080FFFCCF8091D6
:1045900097028093F1008091E8008E778093E80085
:1045A0000C94C124089584B7877F84BF0FB6F89414
:1045B000A8958091600088618093600010926000EF
:1045C0000FBE90E080E80FB6F8948093610090935E
:1045D00061000FBE0C945F200E9413250E94662587
:1045E000E2EEF0E080818460808378940C94CA27A6
:1045F0008EE191E00C94261F8091D0028530A9F4C1
:104600008091D002853079F40E94B1208091CE0251
:104610008823B1F30E947120882391F30E947223B2
:104620000E943A08EDCF0C94DC20089508950C9474
:104630001923292F332723303105C9F060F42130A5
:10464000310581F02230310509F044C08BE390E060
:1046500025EB33E043C021323105E1F02232310550
:1046600049F138C082E190E020EF33E037C099276C
:104670008130910549F028F0029761F5E9E8F3E00F
:1046800005C0E1EBF3E002C0E9E9F3E0849190E0DA
:104690009F0124C06115710541F061307105D1F4AD
:1046A00089E090E020EE33E019C089E090E027EC4B
:1046B00033E014C06115710541F06130710551F4AA
:1046C00086EB90E022E034E009C080E490E028EB43
:1046D00034E004C080E090E020E030E0FA01318373
:1046E0002083089584E089BD86E089BD09B400FE79
:1046F000FDCF8091D8008F7D8093D8008091E0001D
:1047000082608093E0008091E00081FDFCCF0895FD
:10471000CF92DF92EF92FF920F931F93CF93DF938D
:10472000EC018B017A010E94E024811133C0E11475
:10473000F10439F0F70180819181081B190BC80F32
:10474000D91FC12CD12C0115110519F18091E80058
:1047500085FD16C08091E8008E778093E800E11413
:10476000F10449F0F70180819181C80ED91ED182F0
:10477000C08285E00FC00E94E024882321F30AC094
:1047800089918093F10001501109FFEFCF1ADF0AE0
:10479000DACF80E0DF91CF911F910F91FF90EF90E2
:1047A000DF90CF9008952091D7023091D80226173C
:1047B000370748F06115710539F42091E8002E772C
:1047C0002093E80001C0B901FC0120E061157105EA
:1047D00061F18091D0028823D9F18530D9F180919F
:1047E000E80083FD39C08091E80082FD2BC08091F4
:1047F000E80080FFEBCF8091F20090E06115710539
:1048000051F08830910538F421912093F1006150E6
:1048100071090196F3CF21E0089709F020E080911B
:10482000E8008E778093E800D1CF2111D2CF0AC063
:104830008091D002882361F0853061F08091E8009A
:1048400083FD0AC08091E80082FFF2CF80E00895E6
:1048500082E0089583E0089581E008952091D702D1
:104860003091D8022617370748F06115710539F4E1
:104870002091E8002E772093E80001C0B901FC01E7
:1048800020E06115710579F18091D002882309F447
:104890003DC0853009F43CC08091E80083FD3AC0FA
:1048A0008091E80082FD2CC08091E80080FFE9CF74
:1048B0008091F20090E06115710559F08830910502
:1048C00040F424912093F1003196615071090196D2
:1048D000F2CF21E0089709F020E08091E8008E7780
:1048E0008093E800CECF2111CFCF0AC08091D002B3
:1048F000882361F0853061F08091E80083FD0AC073
:104900008091E80082FFF2CF80E0089582E0089570
:1049100083E0089581E00895982F953068F590938D
:10492000E900981739F07091EC002091ED0050915A
:10493000F00003C0242F762F50E021FD02C09F5FBE
:10494000ECCF3091EB003E7F3093EB003091ED00E7
:104950003D7F3093ED003091EB0031603093EB0000
:104960007093EC002093ED005093F0002091EE0046
:1049700027FDE5CF80E008958F708093E90081E006
:1049800008958091D10287FF11C08091E80082FDD7
:1049900005C08091D0028111F8CF11C08091E8004C
:1049A0008B770BC08091D002882349F08091E8007A
:1049B00080FFF8CF8091E8008E778093E80008951B
:1049C0002091E4003091E50095E64091EC00842FC1
:1049D000817040FF23C08091E80080FD1DC0809160
:1049E000D002882399F0853099F08091EB0085FD05
:1049F00011C04091E4005091E5002417350729F3D8
:104A0000915011F09A01E1CF84E0089582E0089579
:104A100083E0089581E0089580E008954091E800E2
:104A200042FFDDCF08950E9470250E947325E0EEBD
:104A3000F0E0808181608083E8EDF0E080818F7715
:104A4000808319BCE3E6F0E080818160808310926E
:104A5000CF0208950E9470250E9473258091D8008E
:104A60008F778093D8008091D80080688093D80099
:104A70008091D8008F7D8093D80084E089BD86E046
:104A800089BD09B400FEFDCF1092D0021092CC0275
:104A90001092CE021092CD0242E060E080E00E94CF
:104AA0008C248091E1008E7F8093E1008091E20070
:104AB00081608093E2008091E20088608093E20050
:104AC0008091E0008E7F8093E0000895E3E6F0E0BF
:104AD00080818E7F808381E08093CF020C942A2591
:104AE0001092E20008951092E10008951F920F9233
:104AF0000FB60F9211242F933F934F935F936F93B1
:104B00007F938F939F93AF93BF93EF93FF93809186
:104B1000E10082FF0BC08091E20082FF07C080911C
:104B2000E1008B7F8093E1000E94C9278091E10022
:104B300080FF19C08091E20080FF15C08091E200E3
:104B40008E7F8093E2008091E20080618093E2009A
:104B50008091D80080628093D80019BC85E0809352
:104B6000D0020E94F3218091E10084FF30C0809147
:104B7000E20084FF2CC084E089BD86E089BD09B4D1
:104B800000FEFDCF8091D8008F7D8093D80080916A
:104B9000E1008F7E8093E1008091E2008F7E809320
:104BA000E2008091E20081608093E2008091CC027B
:104BB000882311F084E007C08091E30087FD02C0E4
:104BC00081E001C083E08093D0020E94FB218091AC
:104BD000E10083FF29C08091E20083FF25C080911E
:104BE000E100877F8093E10082E08093D002109201
:104BF000CC028091E1008E7F8093E1008091E20001
:104C00008E7F8093E2008091E20080618093E200D9
:104C100042E060E080E00E948C248091F000886097
:104C20008093F0000E94F121FF91EF91BF91AF912D
:104C30009F918F917F916F915F914F913F912F91B4
:104C40000F900FBE0F901F9018951F920F920FB6E6
:104C50000F9211242F933F934F935F936F937F9302
:104C60008F939F93AF93BF93CF93DF93EF93FF9374
:104C7000C091E900CF708091EC00D82FD17080FDF9
:104C8000D0E81092E9008091F000877F8093F000D7
:104C900078940E9469261092E9008091F000886063
:104CA0008093F000CD2BCF70C093E900FF91EF917E
:104CB000DF91CF91BF91AF919F918F917F916F9134
:104CC0005F914F913F912F910F900FBE0F901F90CA
:104CD00018951F93CF93DF93CDB7DEB7AA970FB682
:104CE000F894DEBF0FBECDBFE1EDF2E08091F100A0
:104CF000819322E0E93DF207C9F70E9419228091D1
:104D0000E80083FF2EC18091D1029091D202492FF9
:104D100050E04A30510508F024C1FA01EA5BFF4F28
:104D20000C943528803821F0823809F01AC108C067
:104D30008091CD029091CE02992389F082600FC0BC
:104D40008091D5028F70853008F00BC18093E90007
:104D50008091EB0085FB882780F91092E900909103
:104D6000E800977F9093E8008093F1001092F100A3
:104D7000D1C0282F2D7F09F0F4C0882319F082308C
:104D800061F0EFC08091D302813009F0EAC0933026
:104D900009F080E08093CE022EC08091D302811171
:104DA0002AC08091D5028F702FEF280F243008F091
:104DB000D8C08093E9002091EB0020FF1CC0933005
:104DC00021F48091EB00806214C09091EB0090611F
:104DD0009093EB0021E030E0A90102C0440F551F81
:104DE0008A95E2F74093EA001092EA008091EB0086
:104DF00088608093EB001092E9008091E800877F43
:104E00008093E8000E94C124ACC08111AAC0109117
:104E1000D3021F778091E3008078812B8093E30099
:104E20008091E800877F8093E8000E94C1248091F0
:104E3000E80080FFFCCF8091E30080688093E3006E
:104E4000111102C082E001C083E08093D00289C0CA
:104E50008058823008F085C08091D3029091D402AE
:104E60008C3D53E0950779F583E08A838AE2898354
:104E70004FB7F894DE01139620E03EE051E2E32FB5
:104E8000F0E050935700E49120FF03C0E295EF70EB
:104E90003F5FEF708E2F90E0EA3010F0C79601C0B0
:104EA000C0968D939D932F5F243149F74FBF80911A
:104EB000E800877F8093E8006AE270E0CE01019607
:104EC0000E94D32316C06091D5027091D602AE0124
:104ED0004F5F5F4F0E941723BC01892B09F441C02B
:104EE0009091E800977F9093E80089819A810E94D1
:104EF0002E248091E8008B778093E80032C08038C0
:104F000081F58091E800877F8093E8008091CC0252
:104F10008093F1008091E8008E7772CF811121C0DB
:104F20008091D3029091D40299270297D4F4809172
:104F3000E800877F8093E8008091D3028093CC02C1
:104F40000E94C1248091CC02811106C08091E300AF
:104F500087FD02C081E001C084E08093D0020E94FE
:104F600005228091E80083FF0AC08091E800877FD6
:104F70008093E8008091EB0080628093EB00AA961A
:104F80000FB6F894DEBF0FBECDBFDF91CF911F915A
:104F900008950895CF938091D0028823A1F0C09105
:104FA000E900CF709091EC00892F817090FD80E82E
:104FB000C82B1092E9008091E80083FD0E946926C9
:104FC000CF70C093E900CF910895002480FD060EB4
:104FD000660F11F08695D1F7802D0895002455278E
:104FE00004C0080E591F880F991F009729F0769565
:104FF0006795B8F37105B9F7802D952F089587FB54
:10500000082E062687FD819567FD61950E943B2845
:105010000EF4919507FC81950895AA1BBB1B51E1E5
:1050200007C0AA1FBB1FA617B70710F0A61BB70B18
:10503000881F991F5A95A9F780959095BC01CD01BD
:10504000089597FB072E16F4009407D077FD09D03A
:105050000E940D2807FC05D03EF4909581959F4F46
:105060000895709561957F4F0895EE0FFF1F05908D
:10507000F491E02D0994991B79E004C0991F9617CB
:1050800008F0961B881F7A95C9F780950895FC0152
:105090004150504030F001900616D1F73197CF01C2
:1050A0000895882799270895FB01DC0104C08D919C
:1050B0000190801921F441505040C8F7881B990B8A
:1050C0000895F999FECF92BD81BDF89A992780B5D0
:1050D0000895A6E1B0E044E050E00C949B28A8E1DC
:1050E000B0E042E050E00C949B28262FF999FECFC7
:1050F00092BD81BDF89A019700B4021639F01FBA2B
:1051000020BD0FB6F894FA9AF99A0FBE0895039647
:10511000272F0E9476280E947528252F0E94762826
:10512000242F0C9476280196272F0E9476280C9421
:105130007528DC01CB01FC01F999FECF06C0F2BD58
:10514000E1BDF89A319600B40D9241505040B8F745
:065150000895F894FFCF62
:10515600C8001F02280850011E0A14010102000A95
:10516600000A0A0118191A1B1C1D1E1F20215A218C
:105176007D215E21ED21E9215D2101E200E900EAC0
:1051860000B500B600B700CD008301CC008A0192BD
:105196000194012102230224022502260227022A63
:1051A60002B300B4006F007000818283E200E90060
:1051B600EA00B500B600B700CD008301CC008A0135
:1051C60092019401210223022402250226022702CB
:1051D6002A02B300B4006F0070008182833031323E
:1051E600333400010202020206060609090909090A
:1051F600090F0F0F0F0F0F15151518181818181877
:045206001818181844
:00000001FF
